:020000040000FA
:020000001528C1
:08000800200090310B194A257C
:10001000111849268031711E102890319118E2265E
:1000200090319319F72680310900F001F101F201B6
:10003000F301F401F501F601F701F801F901FA0104
:10004000FB01FC01FD01FE01FF0121007830990058
:10005000D9309A00980101309500A0309E00DE3022
:100060008C00F7308D008E0122008C018D018E01F5
:1000700001309D00250001309E00230006308C00D9
:100080008D012400C0308B002100111491149315B0
:1000900020000E108E108E110E080F3922008E00D7
:1000A0002000CC01CD01CE019501980199011E30AF
:1000B000DB004630DA000A30D700D6005B08D800F3
:1000C0005A08D9000C3025009A00980120001C1114
:1000D00028000B309E009C012000FF227E11A831D9
:1000E000DF2080317830A7003230A600B8319C2064
:1000F0008031B53007261430A7004B30A600B83148
:100100009C208031B8300726B530C3250026CC2589
:10011000D5300726B830C325F925CC25D830072699
:1001200009300B26A7000A300B26A600B8319C2008
:100130008031CB3007260B300B26A7000C300B2666
:10014000A600B8319C208031CE30072607300B2620
:10015000A70008300B26A600B8319C208031C130A2
:1001600007268831E824F1248031F22300300B2661
:10017000F20072086039203C0319711001300B261F
:10018000F300B0310B2280310C1002300B26F4004A
:1001900003300B26F50004300B26F60005300B2645
:1001A000F700B83138208031FA117A15FA10FB12B5
:1001B0007B14FC177C1406300B26FD00FD177D1305
:1001C000FD107D1088310427CF2504270C30FC2535
:1001D00004278031B0315927803188311A27803186
:1001E000B83100209031962480317908E039003E02
:1001F000603EF90021003730C70020009831092700
:1002000000208031352900000130E500A130E600F2
:100210009730E700711620308500F03084000230FE
:100220008000840A0030800021002030D000F030AF
:10023000CF002000F9179124F913000000000000FE
:100240002100FF30A4007830A60020009031A024C7
:100250008031000000004030003EF4000330F50023
:100260007908E039093EF90000008B167D1C3C2915
:100270008C1288311D278031FF1F462998317C253B
:1002800088310F2798317C258031FF13711E4D294D
:100290002100911420001C155729210091102000E5
:1002A0001C1D552907309C00572903309C008C19D0
:1002B00075298831042780318C197529FE14DC30AA
:1002C000E4007811F814781490315E2780317B12A5
:1002D0008C1D68297B1A74298831332698311026A1
:1002E00024218031FE1075290723B8310020803188
:1002F000D323FE1C7F29A8319220803136298C1F00
:1003000083290C1B862998310020803179081F39F8
:10031000C900F91B98290319982A013C0319942A4A
:100320004908023C0319902A4908033C0319892A09
:100330004908043C0319822AF91BE2294908053CB3
:1003400003197B2A4908063C0319742A4908083C0A
:1003500003196D2A4908093C0319662A49080A3C11
:1003600003195F2A49080B3C0319582A49080C3C19
:100370000319512A49080D3C03194A2A49080E3C21
:100380000319462A49080F3C0319422A4908103C20
:1003900003193E2A4908113C0319372A4908123C1F
:1003A0000319302A4908133C0319292A4908143C27
:1003B0000319222A4908153C03191B2A4908163C2F
:1003C0000319152A4908173C03190F2AF91BEC29B0
:1003D0004908183C0319082A4908193C0319042A3A
:1003E000F91BA62A49081A3C0319FD29F01BA62A65
:1003F000F0138831CA248031A62AF01B9C2AF013FE
:100400008831BB2480319C2A8831B5248031A62ACA
:10041000F01BA62AF013883192248031A62AF01B03
:10042000A62A883160248031A62AF01BA62A8831AA
:1004300039248031A62AF01BA62AF0138831CD2357
:100440008031A62AF01BA62AF0138831B12380310F
:10045000A62AF01BA62AF013883195238031A62AFC
:10046000F01BA62AF013883182238031A62AF01BC4
:10047000A62AF013883170238031A62A88313523CB
:100480008031A62A8831FA228031A62A8831B72203
:100490008031A62AF01B9C2AF0138831A3228031D8
:1004A0009C2AF01B9C2AF01388318F2280319C2AD1
:1004B000F01BA62AF013883164228031A62AF01B93
:1004C000A62AF013883136228031A62AF01BA62AEC
:1004D000F013883113228031A62AF01BA62A7A173E
:1004E0008831DD218031A62AF01BA62A7A138831B3
:1004F000D5218031A62AF01B9C2AF0138831BC211B
:1005000080319C2AF01BA62AF01388316A218031A1
:10051000A62AF01B9C2AF01388314A2180319C2A9C
:10052000883125258031AA2A883125258031AA2ABB
:10053000883125258031AA2AFB1EA22A903100206D
:10054000AE24803190318E248031AA2A903100204F
:100550002A2080317B1CB02AA83192208031B32A16
:1005600021000E15200079081F39043C031DBB2A09
:1005700090312A208031F91BF82C8C1FD52A0C1FB2
:10058000D52A0D1CCC2A8D1CCC2A0D1DCC2A0D1E63
:10059000CC2A8D1ECC2A7A107A18D52A98311726A3
:1005A0009B21A121A721AD2180317D1FF42AFD1CB3
:1005B000F42A7C083039C9000319F12A103C0319C8
:1005C000ED2A4908203C0319E92A98312924803171
:1005D000F42A983146248031F42A983163248031FA
:1005E000F42A9831822480317C1CFE2A79081F3934
:1005F000043C031DFE2A00300B26F20036290C1E97
:10060000042B71168C12080071128C1608007E10D3
:10061000210021082000A700CB0021002008200095
:10062000A600CA00AC3007268831C6263326002033
:1006300080317723AC30C5238830AF000030AE0066
:100640000030AD00B83106228031A71F2A2B7E145E
:10065000A7132B2B7E10B831F92080312708CB004F
:100660002608CA008831C626803188318730FC25AB
:10067000803177238830A8000030A7000030A60022
:10068000C1239031AF3027258031AC30C523C12341
:100690009031AF301C25362580310D30BF00280841
:1006A000C20013260E30BF002708C20013260F30E9
:1006B000BF002608C20013268831C030FC258031D7
:1006C000280E0F39CE2328080F39CE232030CA2315
:1006D000270E0F39CE2327080F39CE232030CA2307
:1006E000260E0F39CE2326080F39CE2308007E1C94
:1006F0007C2B2D30CA237E2B2030CA234C0E0F3981
:10070000CF00003C031D862BF117892BF1134F08F6
:10071000CE234C080F39CF00003C031D932BF11F53
:10072000932BF117962BF1134F08CE234D0E0F3953
:10073000CF00003C031DA02BF11FA02BF117A32B12
:10074000F1134F08CE234D080F39CF00003C031D95
:10075000AD2BF11FAD2BF117B02BF1134F08CE23AA
:100760004E0E0F39CF00003C031DBA2BF11FBA2BE0
:10077000F117BD2BF1134F08CE234E080F39CE23AE
:100780000800B831932580310800903111254625A5
:100790008031080088310B268031080088316226BC
:1007A0000B26803108009031A2301125B8319C20F1
:1007B000932580310D300B26AF000E300B26AE0096
:1007C0000F300B26AD00B83106229526F920803176
:1007D000200027082100A300200026082100A200F5
:1007E000200008000B2420306F24142425306F24AF
:1007F0001D242A306F2426242F306F242F243430D8
:100800006F24382467306F2441249A306F244A249F
:10081000CD306F24080021002130A9009030A800BD
:100820002030E7002000080021002130A900E0303E
:10083000A8002530E7002000080021002230A90090
:100840003030A8002A30E7002000080021002230C4
:10085000A9008030A8002F30E70020000800210008
:100860002130A9009530A8003430E70020000800AE
:1008700021002130A900E530A8006730E700200002
:10088000080021002230A9003530A8009A30E70086
:100890002000080021002230A9008530A800CD30BA
:1008A000E7002000080021002130D0009530CF0063
:1008B0002000080021002130D000E530CF002000CA
:1008C000080021002230D0003530CF002000080081
:1008D00021002230D0008530CF0020000800BF006A
:1008E0003F080B2689080319792C7B24BF0A85242D
:1008F000702C7B240800C9002100290885002808E5
:10090000840020004908800008002100A80A03197B
:10091000A90A200008002100CF0A0319D00A2000EC
:1009200008002100B630E200ED30E3002000210095
:10093000500885004F088400000820008908031D26
:10094000C42CFE1FAF2CA831002007204720803187
:100950007C1DAE2CFE1FAE2C983133278031A83180
:10096000DE2180317E17FC179831092780319825C8
:10097000031DBE2C9831F2258031C12C98310027FF
:100980008031F0138B1608002100DF00200089035E
:100990000319F02CFE1FD42C210031305F022000FF
:1009A000031DD42C2C25E02C9831162080312100F9
:1009B000E10020007C100B259825031DE02CFC2471
:1009C0007C1CEC2C1818E22C98250319EA2C983181
:1009D000002780318B160800A8257C1CF72CE22C00
:1009E000B0257C18E22C9825031DF72CFC24362911
:1009F0007C18E22C8B24972C22000E302A02031C38
:100A0000AA0A2A08013C20000318092D9831E52480
:100A10008031F0130800210061080739E400063C2A
:100A2000031D142D6111192D6408073C031D192D98
:100A3000E40320002100E1352000031C212DA22524
:100A4000222D9C257C1C272D731E0C1008002100D4
:100A5000E40B192D2000080074083F39CB007508FD
:100A6000CA0085018831C62680314D0E0F39CF006E
:100A70000319442D4F0888316226803163257C108C
:100A80000B25A8257C1808004D080F3988316226EF
:100A9000803163257C100B25A8257C1808004E0E9C
:100AA0000F3988316226803163257C100B25A825FB
:100AB0007C1808004E080F39883162268031632582
:100AC0007C100B250800210061082000CF0073086E
:100AD000E039C90003190800403C0319802D49087A
:100AE000603C03197B2D4908803C0319842D4F0875
:100AF0007D3C03198D2D4F08FD3C0319912D882D48
:100B00004F087D3C03198D2D4F08FD3C0319932D93
:100B10004F08F53C03198F2D08004230942D823088
:100B2000942DE330942D81302100E1002000080055
:100B300079081F39173C0800903120268031701A3F
:100B40009F2D080090312B268031F019A52D08002B
:100B50007011F01470140A305B02D900B825080037
:100B60007011F01070100A305A02D900B825080030
:100B7000711E1C1173121814F0159031FF2480316E
:100B8000F019C02D0800903111256A30272549241D
:100B90006F3011258031080090313E257130AF0053
:100BA0005130AE00B730AD0090313A2590317C30F5
:100BB000AF000F30AE005C30AD003625AC302725DD
:100BC0007F30A800A701A601AC301C253E258F3040
:100BD000AF006A30AE006030AD003A25AC3027255A
:100BE0008E30A800A701A601AC301C253625803127
:100BF00008007830AF001330AE007430AD0008004C
:100C00007830AF003430AE003930AD00080090319C
:100C10002725803108002300910015139513151422
:100C200013082000080042082300930020003F081A
:100C3000230091001513951315158B13553096004D
:100C4000AA30960095149518232E8B1720000800C3
:101000008030FC2508008430FC2508008630FC2553
:1010100008008830FC2508008F30FC250800C0300F
:10102000FC250800C130FC250800C530FC2508005F
:10103000C830FC250800CF30FC250800B230850000
:10104000FA30C2250800B2308500FD30C225080004
:10105000B33085000030C2250800B330850003306E
:10106000C225080020300B2608003E300B26080061
:10107000B2308500EF30C2250800B33085009430CF
:10108000C2250800B33085009830C2250800B3306F
:1010900085009C30C2250800B3308500A230C225EF
:1010A0000800B3308500A630C2250800B3308500A3
:1010B000AC30C2250800B3308500B130C22508002D
:1010C000C830FC25B33085002A30C2250800B33073
:1010D00085003B30C2250800B33085004430C2256E
:1010E0000800CC30FC25B33085003730C22508001D
:1010F000CC30FC25761B8028B33085002130832836
:10110000B33085002530C225080012207F300B2621
:10111000080015207E300B260800B3308500B6305D
:10112000C2250800B33085004930C2250800B3301D
:1011300085007A30C2250800B33085007D30C22595
:101140000800B33085007730C225080031300B2607
:10115000A1207E300B260800B3308500D030C22598
:101160000800B3308500D430C2250800B3308500B4
:10117000DD30C2250800B3308500F930C2250800F3
:10118000B43085000330C22508007408C039C90096
:10119000031DCC288130D9284908403C031DD228A2
:1011A000C130D9284908803C031DD8288830D92867
:1011B000C830FC250E30FC25080079086039C900CC
:1011C00003190729203C0319FD284908403C03194D
:1011D000F3287A1BEF2880312624883108008031DB
:1011E0004A24883108007A1BF92880311D2488316F
:1011F000080080314124883108007A1B032980319E
:1012000014248831080080313824883108007A1B82
:101210000D2980310B248831080080312F2488313A
:101220000800002045300B2679086039C9000319F1
:101230002629203C031924294908403C0319222966
:101240002D20080028200800232008001E20080068
:10125000F8157815F81078103C30E40090315E27CE
:10126000883108004C300B267B183F29B4308500AC
:101270001030C22532203220322032204229B430B0
:1012800085001330C22508000430C900A831F120C0
:1012900088310800FA130725142500201E20B330DA
:1012A00085000630C2250F202320B33085000B3087
:1012B000C22509202820B33085001630C225182009
:1012C0002D20B33085001A30C2250C203520F017B0
:1012D0007B150800FA133326072514250020533008
:1012E0000B261E207408C039031D7829FC147929A7
:1012F000FC1009214421122023207408C039403CED
:10130000031D8429FC148529FC10FF204421092099
:1013100028207408C039803C031D9029FC149129B1
:10132000FC10F520442118202D207408C039C03C41
:10133000031D9C29FC149D29FC10EB2044210C204A
:1013400035207D1FB8297C083039C9000319B5291B
:10135000103C0319B3294908203C0319B129C930AD
:10136000B6298930B629C230B6298230FC2535200D
:10137000C520F0177B150800FA1307251425002057
:1013800045300B261E200921442112202320FF2056
:10139000442109202820F520442118202D20EB206D
:1013A0004421C520F0177B1108008B30FC25B33099
:1013B00085001030C2257B11E0297B150C203520DB
:1013C000FA1707251425852089206020782011210F
:1013D000DD2021006508A8070318A90A290885004F
:1013E00028088400FC1DF629600880002000DD200C
:1013F0007A1BFC290430FD290B30C9002100660846
:10140000A8070318A90A2000A831F120883121007B
:1014100048082000833EFC25F81B112A0E30FC25CD
:101420002821F0170800FA130725142500201E2094
:1014300067200F2023206C20C830FC25B3308500A6
:101440002E30C225CC30FC25B33085003230C22589
:101450008B30FC257E192E2A3220302A63300B2651
:10146000A8312A218831F0177B110800FA130725CB
:101470001425002067208930FC257308E039C90055
:1014800003195E2A203C0319592A4908403C0319D4
:10149000542A32204908603C0319512AA8209C2074
:1014A0005F2AA82097205F2AA62041300B269C2087
:1014B000602AA62041300B269720602A92203220F5
:1014C0007120F0177B110800FA130725142500205E
:1014D000B33085008030C2256C208E30FC25740826
:1014E000C039C9000319872A403C0319832A4908D7
:1014F000803C03197F2AB330850091308A2AB330AB
:1015000085008E308A2AB33085008B308A2AB3302A
:1015100085008830C2257120F0177B110800FA136E
:101520000725142500201E2038200F2023203D20D1
:1015300009202820422018202D2047200C2035206B
:10154000F0177B150800FA130725142500201E202C
:101550004C200F202320562009202820512018201D
:101560002D205B201B203520F0177B150800FA1377
:10157000FA24002038207B08C039C9000319C62A84
:10158000803C0319C42A08001A25F72A1625903131
:10159000D53011256A301C2536258831A71FDA2A57
:1015A000F01B08007C1B0800D5301B25D530E22439
:1015B0007725EC2A90316A301125D8301C25362544
:1015C0008831A71FF32AF01B08007C1B0800D830C5
:1015D0001B25D830E224772598313E218831F01739
:1015E0007C177B1108006A30E224F0137C13772506
:1015F0007B110800FA13FA2400203D207B08C03933
:10160000C9000319092B403C0319272BCB301B259C
:101610002F2B162590316A301125DE301C253625FA
:101620008831A71F292BF01B08007C1B0800DE3027
:101630001B259031DE301125CB30272588317725C9
:1016400098313E218831F0177C177B110800B530A6
:101650001B2590316A301125CB3027258831F013B6
:101660007C13712077257B110800FA13FA240020DF
:1016700042207B08C039C9000319442B403C0319A0
:10168000622BCE301B256A2B16259031DB301125BD
:101690006A301C2536258831A71F642BF01B0800F3
:1016A0007C1B0800DB301B259031DB301125CE3050
:1016B00027258831772598313E218831F0177C170E
:1016C0007B110800B8301B2590316A301125CE30CF
:1016D00027258831F0137C13712077257B110800B2
:1016E000FA1307251425002047200620F61F7B2B20
:1016F00035300B267D2B37300B268D207120F017CF
:101700007B110800FA130725142500204C20062021
:10171000F21F8F2BB3308500BF30C225902B922053
:1017200032207120F0177B110800FA1307251425C9
:1017300000205120062072081F39193EA7000A30E8
:10174000AE00B8315E2088312708CB002608CA00D9
:10175000C62636268A30FC2532207120F0177B11F0
:101760000800FA13072514250020562006207208C9
:1017700060390319C42B203C0319C02BB120C92B9D
:10178000AC20B6203220C92BB3308500CB30C22527
:10179000B6207120F0177B110800FA1307251425D5
:1017A00000205B20062073080F39C9000A3C03198A
:1017B0002D2C49080B3C0319292C3220C908031988
:1017C000252C4908013C0319212C4908023C031926
:1017D0001D2C4908033C0319192C4908043C031922
:1017E000152C4908053C0319112C4908063C03191E
:1017F0000D2C4908073C0319092C4908083C03191A
:10180000052CB43085003B30302CB43085003730A7
:10181000302CB43085003330302CB43085002F307C
:10182000302CB43085002B30302CB430850027307C
:10183000302CB43085002330302CB43085001F307C
:10184000302CB43085001B30302CB430850017307C
:10185000302CB43085004430302CB43085003F301B
:10186000C225B3308500E230C2257120F0177B110C
:101870000800FA13072514250020B3308500E9304D
:10188000C2250F20B3308500EF30C2257820182004
:10189000FA184E2CB3308500F230512CB33085004D
:1018A000F530C225C330FC25B031452188310B26E7
:1018B000B3308500E530C22577257B11F01708008D
:1018C000FA137B15072514257725FC1F832C85200B
:1018D00089200C2035200020DE2421006608A8077E
:1018E0000318A90A6F08A9072000A831F120883140
:1018F000210048082000803EFC25F81B822C0E3079
:10190000FC252821902C0020DE2421006608A80751
:101910000318A90A6F08A9072000A831F12088310F
:10192000F0170800FA13072514250020BB203220E9
:101930001E20B3308500BA30C225152023208D200B
:1019400071208C30FC25FD1FAB2CA8314021883143
:101950008530FC25AF2CA8314021883115200E3070
:10196000FC252821F0177B110800FA130725142500
:1019700077257B110800FA130725142500201E2067
:10198000BB20322025300B260F202320C020F0174B
:101990007B110800FA13072514250020C0208B3086
:1019A000FC25B0315C2188317120F0177B110800D3
:1019B0000020B43085004930C2250800B0310C2128
:1019C0008831080090311125C13027258831080061
:1019D0008031C130C3250026D425DE30072688316A
:1019E00008008031C130C325F925D425DB30072616
:1019F000883108009031B5301125BB302725B8302B
:101A00001125BE302725B8311E20883108009031BD
:101A1000CB301125BB302725CE301125BE302725F0
:101A2000B8311E2088310800FB1E1A2D9031AE24DB
:101A300088310800C13090311125DA24883108003E
:101A4000182032211B2035200800FA13072500201A
:101A500072086039C900C90803193A2D4908203CA9
:101A600003193F2DB12020257908E039F900FB103A
:101A70007B150800B3308500C730C225402DAC204F
:101A8000903100209624883179081F39C900031944
:101A90006F2D013C0319582D4908023C031D080015
:101AA000781B5E2D781398312421883178175E2DAC
:101AB000122038202025FB167B15692D122032209C
:101AC0003220182032203220322032201B203220B7
:101AD0007B110320B2308500F230C225752D032022
:101AE000382020251A25FB127B1577250800903118
:101AF000492488316B08CB006C08CA00C62698318F
:101B000077218831B22579081F39C9000319A92D19
:101B1000013C0319A92D4908023C0319A92D4908C4
:101B20000E3C0319AB2D49080F3C0319AB2D490896
:101B3000103C0319AB2D4908163C0319A92D49087F
:101B4000173C0319A72D4908193C031D080018204C
:101B5000AC2D0920AC2D03203626B2308500F6309E
:101B6000C22508004E0E0F39CE004D0EF039CE07BB
:101B70004D0E0F39CD004C0EF039CD074C0E0F39FC
:101B8000CC000800840080080319CC2D00080B2627
:101B9000840A0319850AC32D8401850108000427DE
:101BA00004273030F42504273030F425FD2630306A
:101BB000F425FD262030F425FD261A262830FC25A4
:101BC0000130FC250630FC2508000E080F39D00036
:101BD0000800F039500422008E00200008008E1505
:101BE00000008E1100000800CF00E5254F08E92510
:101BF0008E100E10EF250800CF00E5254F08E925CF
:101C00008E100E10EF25E5254F0EE9258E100E10D3
:101C1000EF251A260800CF00E5254F08E9258E108C
:101C20000E14EF25E5254F0EE9258E100E14EF2535
:101C30001A26080021000E080F39F03E8E00200001
:101C40000E108E148E1500000E08F039D0008E1183
:101C50000000EF25D01B202E8E1021000E080F391A
:101C60008E00200008000130FC2508004D0E0F39C1
:101C7000CF00031D3F2E7C1D711332204B2E7C198B
:101C8000482E71179831772188314D0E0F39CF00CA
:101C90004F0862260B264D080F3962260B267C1949
:101CA000532E2E300B264E0E0F3962260B267C1932
:101CB0005D2E711F5D2E322008004E080F396226FE
:101CC0000B260800CF00003C031D692EFD30C22604
:101CD00030344F08013C031D702E7D30C226313454
:101CE0004F08023C031D772E3D30C22632344F0888
:101CF000033C031D7E2E1D30C22633344F08043CA6
:101D0000031D852E0D30C22634344F08053C031DBB
:101D10008C2E0530C22635344F08063C031D932E09
:101D20008530C22636344F08073C031D9A2EC53035
:101D3000C22637344F08083C031DA12EE530C226C9
:101D400038344F08093C031DA82EF530C22639341B
:101D50004F080A3C031DAD2E61344F080B3C031D98
:101D6000B22E62344F080C3C031DB72E63344F086B
:101D70000D3C031DBC2E64344F080E3C031DC12EC8
:101D8000653466342100E100200008003F000508AA
:101D9000E90085010408E800200003101030C800A5
:101DA000CC01CD01CE01CA0DCB0DCE0DCD0DCC0D8C
:101DB000C80BE12E3F0069088500680884002000F8
:101DC00000344E308400EB264D308400EB264C303E
:101DD0008400EB26D32E03300007C900C919800008
:101DE00030300007C900C91B800000340730C00034
:101DF00000000000C00BF82E08005130C0000000A9
:101E00000000C00BFF2E08002030C100FF30C000D2
:101E100000000000C00B082FC10B062F08009C30EB
:101E2000C100FF30C00000000000C00B132FC10B29
:101E3000112F08000F270F2708000F270F270F2744
:101E40000F270F270F270F270F270F270F27080010
:102000002100250822003102200003191128210097
:1020100025082200B100210024082200B000200081
:10202000262822003008210024022000043C031846
:10203000080021002408220030022000043C03187C
:102040000800210024082200B00020009831002060
:10205000903108007F2403192F288E2438288424E7
:10206000033C031871288924033C03187128912428
:1020700079081F39C9000E3C0319792849080F3C1B
:10208000031979284908103C031979284908163C96
:1020900003196E284908173C03196E284908193C92
:1020A000031908004908093C031969284908043C38
:1020B000031D7C28F812FB167908E039193EF90057
:1020C0009831FE25903178167C118831B5249031F5
:1020D0000800FB1AAE247E197C280800FB16F013BA
:1020E000080079081F39C900193C0319EF2CFC11AD
:1020F0000800FB137B130800FA1B8228A8319122E9
:1021000090310800FC15761B562A21002508200076
:10211000C500210024082000C400C7012430C600E7
:1021200045247A1E95280230402CC7013630C6005F
:1021300045247A1E9D280330402CC7014830C60034
:1021400045247A1EA5280430402CC7015A30C60009
:1021500045247A1EAD280530402CC7016C30C600DE
:1021600045247A1EB5280630402CC7017E30C600B3
:1021700045247A1EBD280730402CC7019030C60088
:1021800045247A1EC5280830402CC701A230C6005D
:1021900045247A1ECD280930402CC701B430C60032
:1021A00045247A1ED5280A30402CC701C630C60007
:1021B00045247A1EDD280B30402CC701D830C600DC
:1021C00045247A1EE5280C30402CC701EA30C600B1
:1021D00045247A1EED280D30402CC701FC30C60086
:1021E00045247A1EF5280E30402C0130C7000E30F1
:1021F000C60045247A1EFE280F30402C0130C7004F
:102200002030C60045247A1E07291030402C0130AA
:10221000C7003230C60045247A1E10291130402CE8
:102220000130C7004430C60045247A1E19291230F7
:10223000402C0130C7005630C60045247A1E2229A2
:102240001330402C0130C7006830C60045247A1E88
:102250002B291430402C0130C7007A30C6004524A9
:102260007A1E34291530402C0130C7008C30C6004E
:1022700045247A1E3D291630402C0130C7009E307F
:10228000C60045247A1E46291730402C0130C7006D
:10229000B030C60045247A1E4F291830402C01303A
:1022A000C700C230C60045247A1E58291930402C78
:1022B0000130C700D430C60045247A1E61291A3087
:1022C000402C0130C700E630C60045247A1E6A293A
:1022D0001B30402C0130C700F830C60045247A1E60
:1022E00073291C30402C0230C7000A30C600452438
:1022F0007A1E7C291D30402C0230C7001C30C600DD
:1023000045247A1E85291E30402C0230C7002E300D
:10231000C60045247A1E8E291F30402C0230C7008B
:102320004030C60045247A1E97292030402C0230C8
:10233000C7005230C60045247A1EA0292130402C07
:102340000230C7006430C60045247A1EA929223015
:10235000402C0230C7007630C60045247A1EB229D0
:102360002330402C0230C7008830C60045247A1E36
:10237000BB292430402C0230C7009A30C6004524C7
:102380007A1EC4292530402C0230C700AC30C6006C
:1023900045247A1ECD292630402C0230C700BE309D
:1023A000C60045247A1ED6292730402C0230C700AB
:1023B000D030C60045247A1EDF292830402C023058
:1023C000C700E230C60045247A1EE8292930402C97
:1023D0000230C700F430C60045247A1EF1292A30A5
:1023E000402C0330C7000630C60045247A1EFA2967
:1023F0002B30402C0330C7001830C60045247A1E0D
:10240000032A2C30402C0330C7002A30C600452454
:102410007A1E0C2A2D30402C0330C7003C30C600F9
:1024200045247A1E152A2E30402C0330C7004E302A
:10243000C60045247A1E1E2A2F30402C0330C700C8
:102440006030C60045247A1E272A3030402C0330E5
:10245000C7007230C60045247A1E302A3130402C25
:102460000330C7008430C60045247A1E392A323032
:10247000402C0330C7009630C60045247A1E422AFD
:102480003330402C0330C700A830C60045247A1EE4
:102490004B2A3430402C0330C700BA30C6004524E4
:1024A0007A1E542A3530402C0130402C210025085A
:1024B0002000C500210024082000C400C7011230FC
:1024C000C60045247A1E662A3630402CC7012430C7
:1024D000C60045247A1E6E2A3730402CC70136309C
:1024E000C60045247A1E762A3830402CC701483071
:1024F000C60045247A1E7E2A3930402CC7015A3046
:10250000C60045247A1E862A3A30402CC7016C301A
:10251000C60045247A1E8E2A3B30402CC7017E30EF
:10252000C60045247A1E962A3C30402CC7019030C4
:10253000C60045247A1E9E2A3D30402CC701A23099
:10254000C60045247A1EA62A3E30402CC701B4306E
:10255000C60045247A1EAE2A3F30402CC701C63043
:10256000C60045247A1EB62A4030402CC701D83018
:10257000C60045247A1EBE2A4130402CC701EA30ED
:10258000C60045247A1EC62A4230402CC701FC30C2
:10259000C60045247A1ECE2A4330402C0130C700A5
:1025A0000E30C60045247A1ED72A4430402C013014
:1025B000C7002030C60045247A1EE02A4530402C52
:1025C0000130C7003230C60045247A1EE92A463061
:1025D000402C0130C7004430C60045247A1EF22A40
:1025E0004730402C0130C7005630C60045247A1EC3
:1025F000FB2A4830402C0130C7006830C600452413
:102600007A1E042B4930402C0130C7007A30C600B6
:1026100045247A1E0D2B4A30402C0130C7008C30E7
:10262000C60045247A1E162B4B30402C0130C700C3
:102630009E30C60045247A1E1F2B4C30402C0130A2
:10264000C700B030C60045247A1E282B4D30402CE0
:102650000130C700C230C60045247A1E312B4E30EF
:10266000402C0130C700D430C60045247A1E3A2BD6
:102670004F30402C0130C700E630C60045247A1E9A
:10268000432B5030402C0130C700F830C6004524A1
:102690007A1E4C2B5130402C0230C7000A30C60045
:1026A00045247A1E552B5230402C0230C7001C3076
:1026B000C60045247A1E5E2B5330402C0230C700E2
:1026C0002E30C60045247A1E672B5430402C023031
:1026D000C7004030C60045247A1E702B5530402C70
:1026E0000230C7005230C60045247A1E792B56307E
:1026F000402C0230C7006430C60045247A1E822B6D
:102700005730402C0230C7007630C60045247A1E70
:102710008B2B5830402C0230C7008830C60045242F
:102720007A1E942B5930402C0230C7009A30C600D4
:1027300045247A1E9D2B5A30402C0230C700AC3005
:10274000C60045247A1EA62B5B30402C0230C70001
:10275000BE30C60045247A1EAF2B5C30402C0230C0
:10276000C700D030C60045247A1EB82B5D30402CFF
:102770000230C700E230C60045247A1EC12B5E300D
:10278000402C0230C700F430C60045247A1ECA2B04
:102790005F30402C0330C7000630C60045247A1E47
:1027A000D32B6030402C0330C7001830C6004524BE
:1027B0007A1EDC2B6130402C0330C7002A30C60063
:1027C00045247A1EE52B6230402C0330C7003C3094
:1027D000C60045247A1EEE2B6330402C0330C70020
:1027E0004E30C60045247A1EF72B6430402C03304F
:1027F000C7006030C60045247A1E002C6530402C8E
:102800000330C7007230C60045247A1E092C66309A
:10281000402C0330C7008430C60045247A1E122C99
:102820006730402C0330C7009630C60045247A1E1E
:102830001B2C6830402C0330C700A830C60045244C
:102840007A1E242C6930402C0330C700BA30C600F1
:1028500045247A1E2D2C6A30402C0330C700CC3022
:10286000C60045247A1E362C6B30402C0330C7003E
:10287000DE30C60045247A1E3F2C6C30402C0130DF
:102880002100E0002000F013080098315C21903115
:1028900008008E30A800A701A6016A301C25362545
:1028A000AC3027257F30A800A701A601AC301C253D
:1028B0003E258F30AF006A30AE006030AD003A2563
:1028C0007C30AF000F30AE005C30AD00322585307B
:1028D000AF004830AE00AD013A256F30272581307A
:1028E000AF002030AE00AD013A254225A735A63510
:1028F0000318A70A2708EB002608EC0008002100AF
:1029000025082702200008002100260824022000B4
:1029100008002100240826022000080021002508C4
:10292000A70021002408A600200008007F24031926
:10293000A02CF8127908E039023EF9008E24AE2C62
:102940008424073C0318EF2C8924073C0318EF2C40
:10295000F8127908E039023EF9009124A6301125D9
:102960004625AF3027256E30A600A70146258230C8
:10297000AF002030AE00AD013E25AC302725072545
:102980004625AF301C253625AC301C253E25AF3002
:102990001C253225AC30272507254625AF301C25C0
:1029A0003A25AC301C253E25C4301C253A25BE30C6
:1029B0001C2532256A3027257C1B08004225E501AD
:1029C000A735A7350318E50AA6350318A70AA635C3
:1029D0000318A70A2708E6002608E7000800790878
:1029E0001F39C90003190800F81B0800F81A08006D
:1029F0007811F81478105030E4005E27080065085C
:102A0000DD006608DE006708DF00DB260800033013
:102A1000A700FF30A60008000F30A700FC30A6007A
:102A20000800840085010008A80084030008A700AE
:102A300084030008A6000800840085010008AF0098
:102A400084030008AE0084030008AD000800840081
:102A50008501280880008403270880008403260855
:102A600080000800B831082290310800B8310622F1
:102A700090310800B8313E2190310800B8318E21E4
:102A800090310800B831F92090310800B8319C200D
:102A9000903108000B119501FC1F6B2DF91B522D75
:102AA0007D1F932D8C1F752D0C1F752D0D1C612DF9
:102AB0008D1C612D0D1D612D0D1E612D8D1E612D35
:102AC0007A107A18932D0D1C722D8D1C722D0D1DF0
:102AD000722D0D1E722D8D1E702DFC1B932D080066
:102AE000FC1F752D98312421903198315527903154
:102AF00079081F39C900043C03198C2D4908173C7B
:102B00000319872D4908193C03198C2D0800FC175F
:102B10009831092790318F2D983100209031F01293
:102B200070138B1208007E1FA42D2100EA0A031DDA
:102B3000A42DE90A031DA42DE80A681EA42DFD1486
:102B4000E801E901EA017E13711AC12D2100ED0AA5
:102B5000031DB42DEC0A031DB42DEB0A6B1EB42D1E
:102B60007D14EB01EC01ED010E306B02031DC12D54
:102B70003F306C02031DC12D21306D02031DC12D9C
:102B8000FF172000720860392100C500C508200029
:102B90000319E42D210045082000203C0319362E9E
:102BA0001810F21FD62D0C1BDD2DD82D8C1BDD2D02
:102BB0000C14711E1C15731608000C10F81B08006D
:102BC000711E1C1173120800701EF02D711D08007B
:102BD000F21FED2D8C1F701708000C1F70170800D6
:102BE000F01DFC2DF11D0800F21FF92D0C1FF01631
:102BF00008008C1FF0160800F01A202E701B2B2ED8
:102C0000F21F052E0C1F202E072E8C1F202EF21FC8
:102C10000C2E8C1F2B2E0E2E0C1F2B2ED8080319BA
:102C2000142ED708031D08000C10711E1C117312FE
:102C3000D608031D080018107015F0107010080059
:102C40007011F01070140C14711E1C1573161814EA
:102C50007016FF2408007011F01470100C14711E0F
:102C60001C1573161814F015FF240800701A0800BC
:102C7000F0190800F21F3F2E8C1F2B2E412E0C1F27
:102C80002B2EF21F462E0C1F202E08008C1F202EEC
:102C900008001110DC0ADC1C0800DB267208603911
:102CA000203C0319BB2E70080739D300003C0319E0
:102CB000B32E5308013C0319692E5308023C031933
:102CC0007B2ED90B080018100A305B02D900F011D6
:102CD0000800731E8D2E711C722E7119722EE20B5C
:102CE000722E7115D70B08000C10711E1C11731277
:102CF0000A30D7000800731EA02EF11C842EF11993
:102D0000842EE30B842EF115D80B08000C10711ED5
:102D10001C1173125B08D8000800711C942E7119E5
:102D2000942EE20B942E7115D60B0800D2011810C8
:102D30000A30D6006008E20071117012F01208002B
:102D4000F11CA72EF119A72EE30BA72EF115D60B18
:102D50000800D20118100A30D6006108E300F11112
:102D6000F01170130800D90B080018100A305A022D
:102D7000D900F011080070080739013C0319692EC9
:102D8000731ED32EF21FC72E8C1BCE2EC92E0C1BEA
:102D9000CE2E0C14711E1C15731608000C10711E1B
:102DA0001C1173120800D60B0800D20118100A304B
:102DB000D600F01108005D08DC005E0897005F088F
:102DC00096000800911054088700D20A5208283A49
:102DD000031DEB2ED2015208731E003055078600EA
:102DE0000318870A010825009800200008009311A5
:102DF000E40B080028001E119C012000F81378083D
:102E000007392100C6002000023C0319332F21009E
:102E100046082000033C03193F2F210046082000EC
:102E2000043C03194D2F711E1C117312B0310B227B
:102E30009031F01378080739013C031D0800790828
:102E40001F39173C0319252F2A2FF81388316024C6
:102E500090310800FA1F08007A1F0800F813883123
:102E6000DD21903108007908E039781E3B2F043EBF
:102E700078127C153C2F013EF900F81608007B16ED
:102E8000FE1C492F88313326D824983124219031D3
:102E900008009831222090310800F81D552F883104
:102EA0000C30FC259031F8115A2F88310E30FC255A
:102EB0009031F8153C30E4005E27080028001E150C
:062EC0002000F8170800D5
:1030000021000C30EB007330EC009030ED0020001C
:103010007D1008002100510885005F080903520750
:1030200084000318850A00082000080021006208B7
:1030300085005F080903630784000318850A0008F8
:103040002000080079081F39C900FB193728043C03
:103050000319A9284908083C0319C3284908093C51
:103060000319FD284908173C03190E290800031904
:103070009D28013C03199B284908033C03198E280D
:103080004908043C03197D284908083C03197128A4
:1030900049080C3C0319692849080D3C03196128AB
:1030A0004908173C031D08005227173EF900462720
:1030B000FC13F225052788310C30FC25602498315B
:1030C000080052271A3EF90046278831BB24983160
:1030D0009F2852270D3EF90046278831A3229831B8
:1030E0009F28EE257613F2257A135227063EF90023
:1030F00046278831D52198319F28A83100202220E9
:103100009831FE1E85283E210800A8313020472036
:103110009831462788316A2198319F28F926210065
:103120000C14200076135227163EF90046278831EA
:10313000392498319F28FB149E28FB10A1202421BC
:1031400008005227033EF900462788314A2198316A
:1031500008000D1CBB288D1CB7280D1DB3287D173A
:10316000FC167C16BE287D17FC167C12BE287D1727
:10317000FC127C16BE287D17FC127C124627883173
:103180006A21983108000D1CEA288D1CDB280D1CD3
:10319000F3288D1CF328B525031DD428E508031D4D
:1031A000D228D3252000FB28BF25031DD928DB25E5
:1031B000F328CD25D4280D1CF3280D1DF3288F25C9
:1031C0000318FB289925031DE628D325E525A62508
:1031D000DB25F3288D1CF3280D1DF328802503190A
:1031E000FB288525DB250C30E4007811F8147814D1
:1031F00058217B1208003E2108000D1D0929740882
:10320000C039F400F501F50A4627883113229831B8
:103210009F28A831892098317E119F280D1C1C29D8
:103220000D1CF328F4240318FB2800250319FB28A0
:10323000D524E524E025F3288D1CF3280F25031958
:10324000FB281725E025F328711E2D2935309B001A
:10325000B630D4005930D500362921309B002500E6
:10326000113098009A121A1220001C1573160330A0
:10327000E4007811F810781058210800711E4729D1
:10328000FF309B00B430D4005130D50050299F301E
:103290009B002500503098009A121A1220001C152D
:1032A00073160C30E4007811F810781458210800D7
:1032B00090315E27983108004408C602031865293A
:1032C0000130C702031C74296829031D6829FA16F6
:1032D0004508C702031C742903196F297129FA1ABA
:1032E0007229FA127A1600347A12FA1200344E0851
:1032F0000F39043C031808004E08F039103ECE0088
:10330000903C031808004E080F39CE004D08013ECE
:10331000CD000F39093C031808004D08F039103E64
:10332000CD00903C031808004D080F39CD004C0823
:10333000013ECC0008000D1808004B270D180800AE
:10334000B2298D1808004B278D180800B2290D19D5
:1033500008004B270D190800B2290D1A08004B2749
:103360000D1A0800FB11002079081F39C900031944
:10337000B82C013C0319AE2C4908023C0319AB2CB4
:103380004908033C0319912C4908043C0319122CE9
:103390004908053C0319E72B4908063C0319D42BBF
:1033A0004908083C0319872B4908093C03195C2B81
:1033B00049080A3C0319542B49080B3C03194D2BAF
:1033C00049080C3C0319262B49080D3C03190D2B09
:1033D00049080E3C03190A2B49080F3C0319FA2A25
:1033E0004908103C0319EA2A4908113C0319E42A48
:1033F0004908123C0319DE2A4908133C0319D22A52
:103400004908143C0319CA2A4908153C0319BE2A65
:103410004908163C0319872A4908173C03195D2AF5
:103420004908183C03193E2A4908193C03190800A9
:1034300049081A3C0319252AFB19DC2E0D1A08002D
:10344000FD127D12FD117D15FD2DFB19D52E0D1CD4
:103450002E2A8D18080052271B3EFC2D4F270319DA
:10346000352A3E21F81B322AFE2D5227183EF9003C
:1034700046278831922498317A149F28FB19D82E38
:103480000D1C582A8D1C542A0D1A0800FD1F4C2AA9
:1034900077080F39503E4F2A7708F039053EF7007C
:1034A000B831382098315B2AFD1F0800FD135B2AD4
:1034B000FD1B0800FD177C25FE2DFB19F02E0D1CB1
:1034C000772A8D180800FC1F0800F424031C6B2ABF
:1034D0003E21C924080000250319682AD5247C252B
:1034E000E5240126C92477251026E0250800FC1FC5
:1034F00008000F25031D7F2A3E21C32408007C25D8
:1035000017250126C32477251026E0250800FB197E
:10351000E42E0D1CBA2A8D1C9E2A0D1D982A0D1E04
:10352000922A0800761F962A7613FD2D7617FD2D18
:10353000FA1C9C2AFA10FD2DFA14FD2D7A080C397C
:10354000C9000319B02A043C0319AE2A4908083CF3
:103550000319AC2A0030B12A0C30B12A0830B12A44
:103560000430C9007A08F3394907FA00B03145211F
:103570009831FD2DD924C32429250800FB19D12E0B
:103580000D1A08007308F039023EF300B0310B2227
:103590009831FD2DFB19CD2E0D1A08007213F21271
:1035A0001814FD2DFB19CD2E0D1A08007208E039F4
:1035B000053EF200A8319F219831FD2DFB19CD2E3B
:1035C0000D1A0800F213FD2DFB19C52E0D1A080067
:1035D000F613FD2DFB19BD2E0D1A0800FB137B17EA
:1035E0009031B8301125BE3027259831B8311E20D2
:1035F0009831FD2DFB19B52E0D1A0800FB137B1712
:103600009031B5301125BB3027259831B8311E20B7
:103610009831FD2DFB19642E0800FB19632E0D1C3B
:10362000232B8D1C202B0D1D1A2B0D1A0800522741
:10363000153EFC2D4F27031DFA2D5227133EFC2D5E
:103640005227143EFC2D5227123EFC2DFB19472E0B
:103650000D1C432B8D1C3B2B0D1D332B0D1A08000D
:103660005227113EFC2D4F27403C0319FA2D5227BB
:10367000103EF9004A2B4F27403C0319FA2D5227E0
:103680000F3EF9004A2B4F27403C0319FA2D5227D1
:103690000E3EF900FB177B13FD2DFB195C2E0D1A56
:1036A0000800F4137417FD2DFB19582E0D1A08008D
:1036B000F3137313F312FD2DFB19422E0D1C832BF4
:1036C0008D1C7F2B0D1D722B0D1A08007E117C2581
:1036D00001260D1E692B4B270D1E6C2B7B1A3327E1
:1036E000102608007C250126CF247B1E792B33274A
:1036F0000800A8314E2098317E15102608007E1152
:1037000052270B3EFC2D7E1152270A3EFC2DFB1941
:10371000522E0D1CC22B8D1CAB2B0D1D922B0D1E82
:10372000DE2B0800B525031D9D2BE508031D992BF5
:10373000D32520003E21CF240800BF250319A22B4A
:10374000CD259D2B7C257A1FD22B0126CF247725D2
:103750001026DB2508008F25031CB12B3E21C92430
:1037600008009925031DB52BD325E5257C25A62525
:103770007A1FD22B0126C92477251026DB250800C5
:103780003E21FE2D8025031DC82B3E21C3240800A9
:103790007C2585257A1FD22B0126C3247725102668
:1037A000DB2508001026FE2DFB194B2E0D1CE62BE9
:1037B0008D1CE52B0D1DE42B0D1A0800761FE22B46
:1037C0007613FD2D7617FD2D922BAB2BC22BFB19FB
:1037D000472E76130D1C0A2C8D1C022C0D1DFA2B66
:1037E0000D1A0800EE255227083EF9007917F91640
:1037F000F225FD2DEE255227083EF9007917F91222
:10380000F225FD2DEE255227083EF9007913F91611
:10381000F225FD2DEE255227083EF9007913F91205
:10382000F225FD2DFB193E2E0D1C732C8D1C562CE4
:103830000D1D392C0D1A08007A1808007D1F212C47
:10384000772C7C2501260D1A282C7A147B1E232C1C
:1038500010267408C039C03C031D302CFE17312CD3
:10386000FE13F926F9178031682491249831F91351
:1038700008007A1808007D1F3E2C772C7C25012635
:103880000D19452C7A147B1E402C10267408C03963
:10389000803C031D4D2CFE174E2CFE13F926F91704
:1038A0008031612491249831F91308007A180800B6
:1038B0007D1F5B2C772C7C2501268D18622C7A14B9
:1038C0007B1E5D2C10267408C039403C031D6A2CF9
:1038D000FE176B2CFE13F926F91780315A24912418
:1038E0009831F91308007A1808007D1F7A2C7C257E
:1038F000552708007C2501260D18812C7A147B1E83
:103900007C2C10267408C039031D882CFE17892CC6
:10391000FE13F926F9178031532491249831F913B5
:103920000800FB19392E0D1CA52C8D1CA22C0D1D79
:103930009E2C0D1A080052270C3EFC2D7C15522798
:10394000093EFC2D5227053EFC2D7C15F225522701
:10395000043E7A14FC2DFB1908000800FB1908002E
:103960000D1CB52C0D1DBD2C080078135227FC2D05
:10397000FB1908000D1DBD2C08007B1CC12C7B1001
:10398000FD2D7B14FD2D0D1CC32C4B270D1CC62CAF
:1039900008008D1CC92C4B278D1CCC2C08000D1D3C
:1039A000CF2C4B270D1DD22C0800B0310C219831A3
:1039B00008000E275227173EF900FC13FE25F225BA
:1039C0000527883160249831080021000D30480215
:1039D000031CEE2CE60A0319EF0AEF2CC80AE50ACD
:1039E0000319EE0A20000800E925210002306E02CA
:1039F0002000031D080021008F3065022000080010
:103A0000D52421006508A8070318A90A6E08A9078C
:103A1000A80A0319A90A2727000820000800E92599
:103A20002100EE08031D152DE508200008002100E7
:103A3000C808031D212D01306602031CEF03E600B8
:103A4000222DC80301306502031CEE03E5002000AF
:103A500008007C10761B382D652573256525732598
:103A6000803121008D30E10020000B2598313F2D61
:103A7000803121009F30E10020000B259831732513
:103A80007D13F917FE137E13FC1305272100213047
:103A9000D0006030CF002000803191249831F22591
:103AA0007C10F9137325761B5D2D80312100553074
:103AB000E10020000B2598310800803121001530ED
:103AC000E10020000B2598310800803121000430EE
:103AD000E10020000B25A82521004330E100200053
:103AE0000B25983108008031B0259831080051210C
:103AF000711E1C11731208002421F81B7D2D080073
:103B0000E9252100E508200008002100C808031D60
:103B10008B2DE6038C2DC803E50320000800E92562
:103B200021007A1B952D0330962D3130650220003F
:103B30000800E52521006508A8070318A90AA80AB6
:103B40000319A90A272700082000080021007A1B72
:103B5000AB2D0330AC2D0A304802031CB12DE60A10
:103B6000B22DC80AE50A20000800E925E525210054
:103B70006508A8070318A90A2727000808002000DD
:103B8000840A0319850A0008C90001308402031C55
:103B9000850349088000C90808002100A80A031904
:103BA000A90A2727080001308000840A0319850A22
:103BB00000308000080088313326DD21983108006C
:103BC000883133266024983108008831DD2098310F
:103BD000080088310E30FC25983108009031962479
:103BE000983108002100C801E501E601EE01EF016E
:103BF000200008003E21FE2DF900242146277A14DA
:103C0000080079081F39093C0319082E6430092E71
:103C10001E30E4007811F814781458217B12080043
:103C200028001E119C012000F8137B1208008D1A39
:103C300008004B278D1A080000207D1F202E772CAE
:103C4000FB157B1D372E01268D1E242E4B278D1E26
:103C5000272E7B1E372E7C1D2F2E33270800790838
:103C60001F39173C031D0800D924292508001026F8
:103C7000B429EE255227FB18013EFC2D7A180800C6
:103C8000F012442E7E19452E33277C117E114127D8
:103C90005227033EFC2D1227EE257613F2255227DC
:103CA000083EFC2D1227761341275227053EFC2D96
:103CB0000130BF0073085F2E0230BF0074083C273C
:103CC0005227093EFC2DC92E9031C13011254225C5
:103CD000983107302C278831E82498319031CB3047
:103CE0001125DE301C2536259831A71F902E9031E6
:103CF000B5301125DE301C2536259831A71F892EB9
:103D00009031B5301125CB302725DE30272598316D
:103D1000B52E9031DE301125CB3027259831B52EC8
:103D20008831F12498319031DB301125CE301C25BB
:103D300036259831A71FC92E9031DB301125B830B8
:103D40001C2536259831A71FAE2E9031B83011258D
:103D5000CE302725DB3027259831BD2E9031DB3042
:103D60001125CE3027259831BD2E9031CB3011252D
:103D70004225983109302C27C92E9031CE3011259B
:103D8000422598310B302C27C92E0430BF0076080D
:103D90003C277C1352270C3EFC2D0030BF007208DC
:103DA000D42E0130BF0073083C2752270D3EFC2D56
:103DB0000530BF007708DF2E0630BF007D083C27A6
:103DC000412752271A3EFC2D002721000C1020000D
:103DD0008031F2239831761309275227033EFC2DB8
:103DE000FC1BF52EFC170927FD2D41275227163EF7
:103DF000FC2D22007208AB0020007213F2120800A2
:103E000022002B08F200200008002200AA01200056
:103E1000080022000E30AA0020000800B031002067
:103E200098310800E525210067082000BF00210027
:103E3000272720000008C9003C272100E70AA80A1C
:103E40000319A90A2000C908031D132F0800290817
:103E50008500280884000800BF0027083C27BF0A07
:103E600026083C2708000230BF0074083C270330B6
:103E7000BF0075083C270800C20080311326983126
:103E8000080088310C30FC25983108008831332631
:103E90009831F0130800883104279831080072081F
:103EA000603908007908E03908007A147C147D1321
:083EB000F9137E13F013080062
:1050000022007408A2007508A300200008002200F6
:1050100022083F392000C9002200A30A2000031DF6
:105020001228C90A4908273C031D2028220023080A
:105030000F3C20000318202822000F30A30020007E
:105040003E200800220022083F39031D2D28013090
:105050002302031D2D28FE162E28FE122000080014
:1050600022000130A30203183C2822083F39200007
:10507000C9000130C9023E20200008002200220899
:10508000C039200049072200A200200008002200A9
:105090002208F4002308F50020000800220074080C
:1050A0003F39AD007508AC00200008004E202200FA
:1050B000AF012E08AC072F0803182F0AAD072D08E3
:1050C000273C2000031D080022002C080F3C200074
:1050D0000318080022000F30AC00200008004E200A
:1050E0002200AF012E08AC022F08031C2F0AAD02CC
:1050F000031C8328AD082000031D08002200AC0813
:105100002000031D08002200AD010130AC0020008A
:10511000080022007408C0392D07F4002C08F5009F
:1051200020000800903107254625AC302725A43003
:1051300011254625AC301C253625A831A71BA428EF
:1051400090310725A831B7289031B2301C253A2577
:10515000AC30272507254625AC301C2532254225B5
:10516000A8312708033C0318B728A701A601261871
:10517000BD28250013122000C0282500131620008A
:10518000A618C628250093122000C92825009316CA
:105190002000A735A735A735A735A735A735A636EB
:1051A00026362704250091009315131521000E11B2
:1051B00020002800971017101715200008009031C4
:1051C000A7015030A6004625AC302725A701323074
:1051D000A6004625AC301C253E25B2302725A83137
:1051E00008002200AA0820000319080079081F39C6
:1051F000173C031DFF2822002A082000C9002100B7
:1052000029088500280884000008DF00DF08200046
:10521000031929297C1D1829FC1C1829043049026E
:10522000031D1829210031305F02200003192A29AB
:105230002100B630D1008130D200200098310A2000
:10524000A83188310B26A83180318524A831C90BBB
:10525000FF2808007E1D352922002D082000CB00E4
:1052600022002C082000CA003A2974083F39CB00DC
:105270007508CA0085018831C6263626A83108007F
:105280007708FD1F4629F039C90049290F39C9009F
:10529000C90EC9080319982988313220A831490854
:1052A000103C03198F294908203C03198B29490810
:1052B000303C031987294908403C031983294908D0
:1052C000503C03197F294908603C03197B29490890
:1052D000703C031977294908803C03197329B330BE
:1052E000850077309229B330850074309229B3302D
:1052F000850071309229B33085006E309229B33029
:10530000850068309229B330850062309229B3302D
:1053100085005C309229B330850056309229B33035
:10532000850050308831C22525300B26A831080071
:10533000B3308500FE308831C225A83108007208DC
:105340001F39193EDB000800B0310B22A8310800DC
:1053500098315C21A831080079081F39C90008007C
:10536000AC21093C080049080A3C080049080B3CEC
:1053700008004908113C08004908123C0800490887
:10538000133C08004908143C08004908153C080073
:105390004908183C080049081B3C08007208E0391D
:1053A00008007308F03908007708F039080077081A
:1053B0000F390800B8313820A8317C2FFD107D0846
:1053C0003C39C9000319882A043C03197F2A49087B
:1053D000083C0319762A49080C3C03196D2A490830
:1053E000103C0319642A4908143C03195B2A490834
:1053F000183C0319522A49081C3C0319492A490838
:10540000203C0319402A4908243C0319372A49083B
:10541000283C03192E2A49082C3C0319252A49083F
:10542000303C03191C2A21000C30E8007330E900DD
:105430009030EA002000080021000C30E800BF3066
:10544000E9004430EA002000080021000D30E800A7
:105450000A30E900F830EA002000080021000D3091
:10546000E8005630E900AC30EA00200008002100D6
:105470000D30E800A230E9006030EA0020000800AA
:1054800021000D30E800EE30E9001430EA00200081
:10549000080021000E30E8003930E900C830EA0089
:1054A0002000080021000E30E8008530E9007C3043
:1054B000EA002000080021000E30E800D130E900A9
:1054C0003030EA002000080021000F30E8001C30D6
:1054D000E900E430EA002000080021000F30E80075
:1054E0006830E9009830EA002000080021000F3001
:1054F000E800B430E9004C30EA0020000800210048
:105500000F30E800E130E900B830EA002000080080
:1055100021000F30E800F030E900DC30EA00200024
:105520000800210025082000C500210024082000D3
:10553000C400C7015A30C600A8217A1EC72AB0216C
:10554000031DA42A0A30732FB321031DA82AD62BCA
:10555000B621031DAC2A642CB921031DB02A6A2C84
:10556000BC21031DB42A6F2CBF21031DBB2ACE21F1
:10557000F2009F217C2FC221031DBF2A7C2CC52154
:10558000031DC32AB72BC821031D872BFA2BC70184
:105590008730C600A8217A1EF62AB021031DD22A20
:1055A0000930732FB321031DD62AD62BB621031D34
:1055B000DA2A642CB921031DDE2A6A2CBC21031DC2
:1055C000E22A6F2CBF21031DEA2ACE21013EF20000
:1055D0009F217C2FC221031DEE2A7C2CC521031D97
:1055E000F22AB72BC821031D872BFA2BC701B43031
:1055F000C600A8217A1E252BB021031D012B0830DF
:10560000732FB321031D052BD62BB621031D092BA8
:10561000642CB921031D0D2B6A2CBC21031D112BF9
:105620006F2CBF21031D192BCE21023EF2009F21BA
:105630007C2FC221031D1D2B7C2CC521031D212B7A
:10564000B72BC821031D872BFA2BC701E130C600F9
:10565000A8217A1E542BB021031D302B0730732F45
:10566000B321031D342BD62BB621031D382B642CFC
:10567000B921031D3C2B6A2CBC21031D402B6F2C30
:10568000BF21031D482BCE21033EF2009F217C2F1A
:10569000C221031D4C2B7C2CC521031D502BB72B85
:1056A000C821031D872BFA2B0130C7000E30C6001E
:1056B000A8217A1E8C2BB021031D602B0630732F7E
:1056C000B321031D642BD62BB621031D682B642C3C
:1056D000B921031D6C2B6A2CBC21031D702B6F2C70
:1056E000BF21031D782BCE21043EF2009F217C2F89
:1056F000C221031D7C2B7C2CC521031D802BB72BC5
:10570000C821031D842BFA2BCB21031D0800FD1299
:105710007D12FD117D117C2F0130C7003B30C6008A
:10572000A8217A1EC72BB021031D982B0530732F9B
:10573000B321031D9C2BD62BB621031DA02B642C5B
:10574000B921031DA42B6A2CBC21031DA82B6F2C8F
:10575000BF21031DB02BCE21053EF2009F217C2FDF
:10576000C221031DB42B7C2CC521031DBB2BD121D1
:10577000F300A4217C2FC821031DBF2BFA2BCB21C2
:10578000031D0800FD127D12FD117D157C2F0130D7
:10579000C7006830C600A8217A1E0D2CB021031D59
:1057A000D32B0430732FB321031DDA2BF3137313A0
:1057B000F3127C2FB621031DDE2B642CB921031DAF
:1057C000E22B6A2CBC21031DE62B6F2CBF21031D8D
:1057D000EE2BCE21063EF2009F217C2FC221031D1D
:1057E000F22B7C2CC521031DFA2BD121013EF300A5
:1057F000A4217C2FC821031D052CFD1F022CD721BD
:10580000F700DA29D421F700DA29CB21031D08009B
:10581000FD127D12FD157D117C2F0130C7009530E2
:10582000C600A8217A1E4E2CB021031D192C03306E
:10583000732FB621031D1D2C642CB921031D212CAF
:105840006A2CBC21031D252C6F2CBF21031D2D2C80
:10585000CE21073EF2009F217C2FC221031D312C57
:105860007C2CC521031D392CD121023EF300A4213B
:105870007C2FC821031D462CFD1F422CD721103E32
:10588000F700DA29D421013EF700DA29CB21031DE4
:105890000800FD127D12FD157D157C2F0130C7001B
:1058A000C230C600A8217A1E9D2CB021031D5A2C9F
:1058B0000230732FB321031D612CF3137313F316FE
:1058C0007C2FB621031D672CF41374137C2FB92190
:1058D000031D6C2CF6177C2FBC21031D712CF213B9
:1058E0007C2FBF21031D792CCE21083EF2009F2181
:1058F0007C2FC221031D802C7213F21218147C2FEE
:10590000C521031D882CD121033EF300A4217C2F47
:10591000C821031D952CFD1F912CD721203EF70097
:10592000DA29D421023EF700DA29CB21031D080031
:10593000FD127D16FD117D117C2F0130C700EF3067
:10594000C600A8217A1ECE2CB021031DA92C01303F
:10595000732FBF21031DB12CCE21093EF2009F21E0
:105960007C2FC521031DB92CD121043EF300A421B5
:105970007C2FC821031DC62CFD1FC22CD721303E11
:10598000F700DA29D421033EF700DA29CB21031DE1
:105990000800FD127D16FD117D157C2F0230C70019
:1059A0001C30C600A8217A1E1D2DB021031DDA2C43
:1059B0004E207C2FB321031DE12CF3137317F31238
:1059C0007C2FB621031DE72CF41374177C2FB9210B
:1059D000031DEC2CF6137C2FBC21031DF12CF217B8
:1059E0007C2FBF21031DF92CCE210A3EF2009F21FE
:1059F0007C2FC221031D002D7213F21618147C2F68
:105A0000C521031D082DD121053EF300A4217C2FC3
:105A1000C821031D152DFD1F112DD721403EF70074
:105A2000DA29D421043EF700DA29CB21031D08002E
:105A3000FD127D16FD157D117C2F0230C700493007
:105A4000C600A8217A1E562DB021031D292D013034
:105A5000782FB921031D2D2DEA2CBC21031D312DDA
:105A6000EF2CBF21031D392DCE210B3EF2009F21CB
:105A70007C2FC521031D412DD121063EF300A42119
:105A80007C2FC821031D4E2DFD1F4A2DD721503ECE
:105A9000F700DA29D421053EF700DA29CB21031DCE
:105AA0000800FD127D16FD157D157C2F0230C70004
:105AB0007630C600A8217A1EA32DB021031D622DC9
:105AC0000230782FB321031D692DF3137317F316DA
:105AD0007C2FB621031D6F2DF41774137C2FB92171
:105AE000031D732DEA2CBC21031D772DEF2CBF2144
:105AF000031D7F2DCE210C3EF2009F217C2FC22161
:105B0000031D862D7217F21218107C2FC521031D5C
:105B10008E2DD121073EF300A4217C2FC821031D27
:105B20009B2DFD1F972DD721603EF700DA29D42148
:105B3000063EF700DA29CB21031D0800FD167D1271
:105B4000FD117D117C2F0230C700A330C600A821B3
:105B50007A1EE02DB021031DAF2D0330782FB9211F
:105B6000031DB32DEA2CBC21031DB72DEF2CBF2143
:105B7000031DBF2DCE210D3EF2009F217C2FC2219F
:105B8000031DC32D822DC521031DCB2DD121083E20
:105B9000F300A4217C2FC821031DD82DFD1FD42D77
:105BA000D721703EF700DA29D421073EF700DA2921
:105BB000CB21031D0800FD167D12FD117D157C2FE4
:105BC0000230C700D030C600A8217A1E2A2EB0218C
:105BD000031DEC2D0430782FB321031DF32DF31793
:105BE0007313F3127C2FB621031DF92DF4177417CC
:105BF0007C2FB921031DFD2DEA2CBC21031D012E94
:105C0000EF2CBF21031D092ECE210E3EF2009F2155
:105C10007C2FC221031D0D2E822DC521031D152EA3
:105C2000D121093EF300A4217C2FC821031D222E7F
:105C3000FD1F1E2ED721803EF700DA29D421083E11
:105C4000F700DA29CB21031D0800FD167D12FD1592
:105C50007D117C2F0230C700FD30C600A8217A1EBE
:105C60006F2EB021031D362E0530782FB321031D72
:105C70003A2EEF2DB621031D3E2EF62DB921031D20
:105C8000422EEA2CBC21031D462EEF2CBF21031D02
:105C90004E2ECE210F3EF2009F217C2FC221031DEC
:105CA000522E822DC521031D5A2ED1210A3EF3000A
:105CB000A4217C2FC821031D672EFD1F632ED72131
:105CC000903EF700DA29D421093EF700DA29CB21EA
:105CD000031D0800FD167D12FD157D157C2F033078
:105CE000C7002A30C600A8217A1EAB2EB021031DA2
:105CF0007B2E0630782FB321031D7F2EEF2DB6218A
:105D0000031D832EF62DB921031D872EEA2CBC21FD
:105D1000031D8B2EEF2CBF21031D932ECE21103E91
:105D2000F2009F217C2FC221031D972E822DC521B9
:105D3000031D9F2ED1210B3EF300A4217C2FC821EF
:105D4000031DA32E5A2ECB21031D0800FD167D1620
:105D5000FD117D117C2F0330C7005730C600A821EC
:105D60007A1EE32EB021031DB72E0730782FB32102
:105D7000031DBB2EEF2DB621031DBF2EF62DB9211D
:105D8000031DC32EEA2CBC21031DC72EEF2CBF21FF
:105D9000031DCF2ECE21113EF2009F217C2FC22168
:105DA000031DD32E822DC521031DD72E9A2EC82167
:105DB000031DDB2E5A2ECB21031D0800FD167D1678
:105DC000FD117D157C2F0330C7008430C600A8214B
:105DD0007A1E132FB021031DEF2E0830782FB32128
:105DE000031DF32EEF2DB621031DF72EF62DB9213D
:105DF000031DFB2EEA2CBC21031DFF2EEF2CBF211F
:105E0000031D072FCE21123EF2009F217C2FC221BD
:105E1000031D0B2F822DC521031D0F2F9A2EC82184
:105E2000031DDE2E5A2E0330C700B130C600A82154
:105E30007A1E432FB021031D1F2F0930782FB32165
:105E4000031D232FEF2DB621031D272FF62DB9217A
:105E5000031D2B2FEA2CBC21031D2F2FEF2CBF215C
:105E6000031D372FCE21133EF2009F217C2FC2212C
:105E7000031D3B2F822DC521031D3F2F9A2EC821C4
:105E8000031DDE2E5A2E0330C700DE30C600A821C7
:105E90007A1E0800B021031D4F2F0A30782FB3213E
:105EA000031D532FEF2DB621031D572FF62DB921BA
:105EB000031D5B2FEA2CBC21031D5F2FEF2CBF219C
:105EC000031D672FCE21143EF2009F217C2FC2219B
:105ED000031D6B2F822DC521031D6F2F9A2EC82104
:105EE000031DDE2E5A2E2200AE0020006F207C2FD4
:0C5EF0002200AE0020005620F013080035
:10600000FE11803104300B263F39C9007608C039B3
:106010004907F600B03176083F3915062200A10085
:10602000A0012000A7012200290820000739A600AE
:10603000903146256F301C253A25AC302725A70125
:106040000530A6004625AC301C253A25AC30272566
:10605000B03113219031AC301C253625B031A71F4B
:106060003328132136289031AC3011259031422548
:106070002708CB002608CA008831C6260230C8008F
:10608000983177218831B225B031C80B4028D92109
:106090000130CA02031CCB034B082200A7002000DA
:1060A0004A082200A80020000C212200FA1C5A28CD
:1060B000A4015C280530A40020002D212200A208A4
:1060C000200003195D28FA186B28220022082000FE
:1060D000013C03195D28761F6F284C3070283E3034
:1060E00022002202031C7628A2006B28A2082000AE
:1060F00003195D28FA188228220022082000013C9A
:1061000003195D28761BB328220022082000313CA9
:1061100003195D28220022082000333C03195D2862
:10612000220022082000353C03195D28031CA72803
:10613000FA1CC928220022032000031DA528FE1DE9
:106140005D287E1A5D287E16C9287E12C928FA1C91
:106150005D28FE1D5D287E1A5D287E160130220016
:10616000A2002000C92822002208013C031DB928F2
:106170009F28393022020318C1283430A2077E122A
:10618000C928433022020318A7281D30A2027E121C
:10619000C92822002208200080317B248524B031C8
:1061A0002200FA18E528A40BE5280530A4000130E8
:1061B000A8020318DF280130A702031CF8282000DA
:1061C000013080317B248524B03121002330290225
:1061D000031DEE28EF3028020319F828FE152200CF
:1061E0000130A80203185D280130A70203185D28BA
:1061F0002000003080317B24B0317608C039F600B1
:10620000220021083F392000F6060430BF0076083E
:1062100098313C27B031080021002130A9006030BE
:10622000A8002000080090317F30A700FF30A600B2
:106230004625AF302725A7010230A6004625AF30FE
:106240001C253A25AF302725A7010130A600462599
:10625000AF301C253225B031080022002108A300F0
:106260002008A2000310A10DA00D2108A3072008FB
:106270000318200AA2077930A3070318A20A2308EB
:10628000A0002208A100200008007A080C39C900EB
:1062900003195729043C031955294908083C0319D7
:1062A0005329343058293330582932305829313065
:1062B0002200A900200008007D083C39C90003190C
:1062C000C729043C0319C3294908083C0319BF29FD
:1062D00049080C3C0319B8294908103C0319B42992
:1062E0004908143C0319B0294908183C0319AC2982
:1062F00049081C3C0319A8294908203C0319A42972
:106300004908243C0319A0294908283C03199C2961
:1063100049082C3C031998294908303C0319942951
:10632000B33085006E30BB29B33085006B30BB299C
:10633000B33085006830BB29B33085006530BB2998
:10634000B33085006230BB29B33085005F30BB2994
:10635000B33085005C30BB29B33085005930BB2990
:10636000B33085005630BB29B33085005330BB298C
:10637000B330850050308831C225B031CA29D121CF
:106380003530D521CA29D1213230D521CA29D12190
:106390003130D521B43085000C308831C225B03180
:1063A000080088313220B031080088310B26B03126
:1063B0000800CB014C080F39CA00EE214D0EEA212E
:1063C0004D08EA214E0EEA214E080F39CA0703187C
:1063D000CB0A00340F39CA070318CB0A03104A0D41
:1063E0002200A60020004B0D2200A5002000031073
:1063F000CA0DCB0D0310CA0DCB0D0310CA0DCB0D6A
:10640000220026082000CA070318CB0A220025080C
:106410002000CB07003473080F39D3000319462A34
:10642000013C0319552A5308023C0319642A5308F6
:10643000033C0319732A5308043C0319822A5308A6
:10644000053C0319912A5308063C0319A02A530856
:10645000073C0319AF2A5308083C0319BE2A530806
:10646000093C0319CD2A53080A3C0319DC2A711E82
:106470003F2AB630D4003130D5005E30ED2A3B30B3
:106480009B0025009A121A121E30EA2A711E4E2A0B
:10649000B430D4007930D500C730ED2A7C309B0071
:1064A00025009A161A123E30EA2A711E5D2AB4306F
:1064B000D400A130D500B530ED2A71309B00250005
:1064C0009A121A123930EA2A711E6C2AB430D4009A
:1064D000C930D500A630ED2A67309B0025009A12FE
:1064E0001A123430EA2A711E7B2AB430D400F130FB
:1064F000D5009930ED2A5F309B0025009A121A12C0
:106500003030EA2A711E8A2AB530D4001930D500FD
:106510008E30ED2A58309B0025009A161A122C3026
:10652000EA2A711E992AB530D4004130D500843052
:10653000ED2A52309B0025009A161A122930EA2AB9
:10654000711EA82AB530D4006930D5007C30ED2A00
:106550004D309B0025009A121A122730EA2A711E2C
:10656000B72AB530D4009130D5007530ED2A4930C6
:106570009B0025009A121A122530EA2A711EC62A9B
:10658000B530D400B930D5006E30ED2A44309B00D0
:1065900025009A161A122230EA2A711ED52AB53021
:1065A000D400E130D5006830ED2A41309B00250051
:1065B0009A121A122130EA2A711EE42AB630D40047
:1065C0000930D5006330ED2A3E309B0025009A1635
:1065D0001A121F309800200008009B0008004D345C
:1065E0007934003456346F346C340034773470347A
:1065F0006D34003431343A34003432343A340034B7
:1066000033343A34003434343A3400345334453477
:106610004E34443400344534443449345434003422
:106620007434693474346C34653400343034303448
:10663000313400344334573420344B3445345934E6
:10664000003441342D345A340034DC34CC34DE345C
:10665000DD340034443445344C340034433448345D
:1066600047340034313443344C34523400344434ED
:106670004534463400344E346F342E34533474343D
:1066800079346C346534003454347234693467348A
:1066900000344E344F3452344D3441344C34003491
:1066A0003134303400343134353400343234303421
:1066B000003432343534003433343034003433343D
:1066C0003534003434343034003434343534003428
:1066D00035343034003435343534003436343034E5
:1066E0000034373430340034383430340034393402
:1066F000303400344E344F3400344E34543400348B
:1067000043346E347434203475347034203400349F
:106710004D34313400344D34323400344D3433345C
:1067200000344D34343400344D3461347834003422
:106730004D3469346E34003453345034413443346E
:106740004534003450346F346C3400345234613486
:10675000743469346F3400345434793470346534AB
:10676000003454346F346E346534003464346F3420
:106770007434003464346134733468340034523413
:10678000453456344534523453344534003445345A
:106790004C344534003445344C34453443340034AF
:1067A0004234553447340034533454345234413431
:1067B000493447344834543400342D344B34453450
:1067C0005934003448347A3400346D3469346E34CA
:1067D000003454347234613469346E3400344734D4
:1067E0006F34003435344C34003452344E34443435
:1067F00000344D3465346D346F3400346E346F348E
:106800006E3465340034523450345434203474348B
:1068100069346D3465340034733465346334003462
:106820006F346E3400346F3466346634003435347B
:106830003034303400343534353430340034363488
:106840003034303400343634353430340034373476
:106850003034303400343734353430340034383464
:106860003034303400343834353430340034393452
:106870003034303400343934353430340034313449
:106880003034303430340034313430343534303412
:106890000034443449344D342034413464346A344F
:1068A00000347F349334A634B934CA34D934E6344E
:1068B000F034F834FC34FE34FC34F834F034E6348C
:1068C000D934CA34B934A63493347F346B34583451
:1068D00045343434253418340E340634023400344C
:1068E000023406340E3418342534343445345834E4
:1068F0006B3463347234823490349D34A934B334AD
:10690000BB34C134C534C634C534C134BB34B334EC
:10691000A9349D3490348234723463345434443412
:10692000363429341D3413340B3405340134003427
:10693000013405340B3413341D34293436344434D3
:1069400054345A346834763483348F349A34A334CC
:10695000AA34B034B334B434B334B034AA34A33426
:106960009A348F348334763468345A344C343E3419
:10697000313425341A3411340A34043401340034E7
:10698000013404340A3411341A34253431343E3499
:106990004C34533460346D34793484348E349634CA
:1069A0009D34A234A534A634A534A2349D34963443
:1069B0008E34843479346D3460345334463439340D
:1069C0002D342234183410340934043401340034A2
:1069D0000134043409341034183422342D34393459
:1069E00046344C34583463346F34793482348934C7
:1069F0009034943497349834973494349034893460
:106A0000823479346F34633458344C344034353400
:106A100029341F3416340F3408340434013400345C
:106A20000134043408340F3416341F342934353417
:106A30004034473452345D346734713479348034AF
:106A400086348B348D348E348D348B34863480345C
:106A50007934713467345D34523447343C343134E2
:106A600027341D3415340E34083403340134003413
:106A70000134033408340E3415341D3427343134D2
:106A80003C3442344C345634603469347134773495
:106A90007D34813483348434833481347D34773459
:106AA00071346934603456344C34423438342E34C2
:106AB00024341B3413340D340734033401340034CC
:106AC0000134033407340D3413341B3424342E348E
:106AD00038343E34483451345A3462346A34703471
:106AE000753479347B347C347B3479347534703448
:106AF0006A3462345A34513448343E3434342B349A
:106B000022341A3412340C34073403340134003480
:106B10000134033407340C3412341A3422342B3445
:106B200034343A3443344C3454345C34633469344C
:106B30006E34713473347434733471346E34693434
:106B400063345C3454344C3443343A343134283470
:106B50002034183411340B34063403340134003437
:106B60000134033406340B341134183420342834FF
:106B70003134373440344834503457345E3463341D
:106B800068346B346D346E346D346B346834633414
:106B90005E34573450344834403437342E3426343D
:106BA0001E34173410340B340634033401340034EB
:106BB0000134033406340B34103417341E342634B5
:106BC0002E3434343C3444344C34533459345E34ED
:106BD00062346534673468346734653462345E34F3
:106BE000593453344C3444343C3434342C34243409
:106BF0001C3415340F340A340634033401340034A1
:106C00000134033406340A340F3415341C3424346C
:106C10002C3431343934403447344E3454345934BC
:106C20005D34603461346234613460345D345934CD
:106C300054344E34473440343934313429342234D6
:106C40001B3414340E340934053402340134003456
:106C500001340234053409340E3414341B34223424
:106C600029342F3436343E3444344B345034553484
:106C700059345C345D345E345D345C34593455349D
:106C800050344B3444343E3436342F34283420349A
:106C90001A3413340E340934053402340134003408
:106CA00001340234053409340E3413341A342034D8
:106CB00028341A341E342234263429342C342F3408
:106CC00031343334343434343434333431342F3491
:106CD0002C342934263422341E341A341634123417
:106CE0000E340B34083405340334013400340034DA
:106CF000003401340334053408340B340E341234B8
:106D00001634203441344234433444344534463418
:106D10004734483449344A344B344C344D344E347F
:106D20004F3450345134523453345434553456342F
:106D30005734583459345A34313432343334343487
:106D40003534363437343834393430342E342C3406
:106D50003A343F3427342D34283429342F34403406
:106D600022342A343D3404342B340534B134B23463
:106D7000B334B434B534B634B734B834B934BA34BF
:106D8000BB34BC34BD34BE34BF34C034C134C2346F
:106D9000C334C434C534C634C734C834C934CA341F
:106DA000CB34CC34CD34CE34CF34D034D134D234CF
:106DB000D334D434D534D634D734D834D934DA347F
:106DC000DB34DC3401340234A634DD34DE34DF3429
:106DD000B0340334A234A334A434FF3442348434B2
:106DE000A434833401342434C3340434023474347A
:106DF000A3344434C2348234E3346434D43443346A
:106E0000033481342334143463349434B434C434B8
:106E10007D343D341D340D3405348534C534E534BA
:106E2000F534FD345734CF34E63436347E34873489
:106E3000B534B73495346E344E34FF348D34173452
:106E40005534B534DD3442342334BD344534443410
:106E5000A5341434B434F434AD34D534ED3475344D
:106E6000E4348234243464345D3425344334A4342B
:106E70000434D43434348434CD34C43401348334CD
:106E800094342D3481348D34953463349D34C2343C
:106E90000334C334B534E3345434A3344D3465344B
:106EA00074345534023435346D345634B7344E347A
:106EB000573488314830FC2502300B2602300B262F
:106EC0001F300B260A300B261F300B2602300B26F4
:106ED00002300B2600300B265030FC2500300B26EC
:106EE0001F300B2601300B2605300B2606300B26F3
:106EF00004300B261F300B2600300B265830FC25A3
:106F000000300B2600300B2600300B2600300B26FD
:106F100000300B2610300B261F300B2600300B26BE
:106F20006030FC2512300B2614300B2619300B264E
:106F300013300B2605300B260F300B2611300B2695
:106F400000300B266830FC2514300B2618300B2639
:106F500014300B261B300B260D300B260B300B2666
:0C6F600009300B2600300B26B031080071
:107000000530112021001C08A5001B08A400200049
:107010000930112021001C08A1001B08A00020003D
:10702000080021009D0020008831F626F626B831A0
:1070300021009D149D181A28200008009031072572
:107040004625AC3027257F30A800A701A601AC302B
:107050001C253E25AC302725BB301125BE301C2514
:107060003625AC301C253A25C4302725B831080018
:107070000A30A700A735770E0F39AE00AE08031D02
:10708000432871104428711459202608E000E200BA
:107090005B080A3EA70077080F39AE00AE08031D53
:1070A0005328F1105428F11459202608E100E30078
:1070B00008005E200A30AE0073200800A6010830E8
:1070C000B4002708AE0C03186928B40B6228A70186
:1070D000003403106E28AE0C0318A707A70CA60CEB
:1070E000B40B6B280034A3010830B400270DA30DA6
:1070F0002E08A30203187E28A3070310A70DB40BC4
:107100007628B3010830B400260DA30DB30D2E0868
:10711000A302A2010301031C220FB3020318982843
:107120002E08A307A20103010318220FB3070310BF
:10713000A60DB40B842800348E30A8002708A900BF
:10714000A71FA728A609A709A60A0319A70AB3011A
:107150002708031DB1282608A7000319C128A60186
:10716000B3153308A802031D031CFA290310A71B3B
:10717000BE28A60DA70DA80BB728FA29A91FA7138B
:107180000034A701A601A501A8010034B301270816
:10719000031DDB282608A7002508A600A501B315B6
:1071A0002708031DDB282608A700A601B311331604
:1071B00027080319C1283308A802031D031CFA2954
:1071C0000310A71BE928A50DA60DA70DA80BE12804
:1071D000FA292A1B261CBE28A51FBE28A60A0319A9
:1071E000A70A031DBE28A70CA60CA80A0319842908
:1071F000BE282808031900342708A900A7178E30D5
:10720000A802A81F3329A809A80A08302802031CCD
:107210001929A800A60D2708A600A70108302802F2
:10722000031C1929A800A60DA6012808031D031098
:1072300021292808031921290310A70CA60CA80B43
:107240001C292A1B261C2B29031C2B29A60A0319DF
:10725000A70AA71B3329A91F0034A609A709A60A54
:107260000319A70A00342A14AA1FFF34A701A91F73
:10727000FF30A700A600A90DA70CFF342808031DA6
:107280002F080319C12827082E06A9002F08A807D0
:107290007E30031C4F29A802031884295229A80212
:1072A000031CFA292708A5002608A400A517AE1775
:1072B0000310A701A6011030B300241C65292D0876
:1072C000A6072E0803182E0FA707A70CA60CA50CBF
:1072D000A40C0310B30B5D29A71B7229A50DA60DE5
:1072E000A70DA8032A1B261C8129A51F8129A60AF0
:1072F0000319A70A031D8129A70CA60CA80A0319C4
:107300008429A91FA7130034AA14AA1FFF34FF3031
:10731000A800A700A600A90DA70CFF342F08031989
:10732000042A28080319C12827082E06A900A71730
:10733000AE17B3012708A5002608A4002D08A40253
:107340002E08031C2E0FA502A501A401031CAE29C3
:107350000310A70CA60CA50C0130B3002F08A8023F
:10736000031CB8297E303307A80703188429BD29D8
:107370007E303307A807031CFA291030B200A40D91
:10738000A50DA60DA70DB30D2D08A6022E08031CF2
:107390002E0FA7022E0DB304331CD0292414D72995
:1073A0002D08A6072E0803182E0AA7072410B20BD3
:1073B000BF292A1B241CF3290310A60DA70DB30D0A
:1073C0002D08A6022E08031C2E0FA7022E0D330433
:1073D0000139A4070318A50A031DF329A50CA40C61
:1073E000A80A03198429A91FA5132508A7002408A2
:1073F000A60000342A15AA1FFF340130A800A701F7
:10740000A601A90DA70CFF34AA15FF348030AE06E3
:1074100027082E06B300A501AC0128082F02031C83
:10742000232A2F08A3002808AF002308A8002E084D
:10743000A3002708AE002308A7002D08A3002608F4
:10744000AD002308A6002F08031900342708A9005F
:10745000A717AE172F082802AF000319492A0830D2
:107460002F02031C402AAF002D08AC002E08AD00EF
:10747000AE0108302F02031C402A2908A70000345F
:107480002F080319492A0310AE0CAD0CAC0CAF0B3E
:10749000432AB31F532AAC09AD09AE09AC0A03193C
:1074A000AD0A0319AE0A2C08A5072D0803182D0FE5
:1074B000A6072E0803182E0FA707B31B672A031C65
:1074C000E928A70CA60CA50CA80FE9288429031805
:1074D000C628A509A609A709A50A0319A60A03191A
:1074E000A70A8030A906A728B3012708031D892A07
:1074F0002608A7002508A600A501B3152708031D27
:10750000892A2608A700A601B311331627080319F4
:107510009A2A3308A802031D031CC82B0310A71BBB
:10752000972AA50DA60DA70DA80B8F2AC82BA91F5A
:10753000A7130034A701A601A501A401A8010034E6
:10754000B3012708031DC02A2608A7002508A600A6
:107550002408A500A401B3152708031DC02A260886
:10756000A7002508A600A501B31133162708031D9F
:10757000C02A2608A700A601B315270803199A2ACE
:107580003308A802031D031CC82B0310A71BCF2A16
:10759000A40DA50DA60DA70DA80BC62AC82B2A1B46
:1075A000251C972AA41F972AA50A0319A60A0319BE
:1075B000A70A031D972AA70CA60CA50CA80A031955
:1075C000352B972A2808031D2F0803199A2A270804
:1075D0002E06A9002F08A8077E30031CF32AA80254
:1075E0000318352BF62AA802031CC82B2708A40071
:1075F0002608A3002508A200A417AE170310A701B0
:10760000A601A5011830B300221C102B2C08A507D9
:107610002D0803182D0FA6072E0803182E0FA707F5
:10762000A70CA60CA50CA40CA30CA20C0310B30B66
:10763000042BA71B202BA40DA50DA60DA70DA80399
:107640002A1B251C322BA41F322BA50A0319A60ABC
:107650000319A70A031D322BA70CA60CA50CA80A18
:107660000319352BA91FA7130034AA14AA1FFF342E
:10767000FF30A800A700A600A500A90DA70CFF34A5
:107680002F080319D32B280803199A2A27082E0636
:10769000A900A717AE17B3012708A4002608A30066
:1076A0002508A2002C08A2022D08031C2D0FA302FE
:1076B0002E08031C2E0FA402A401A301A201031C87
:1076C000682B0310A70CA60CA50CA40C0130B3006A
:1076D0002F08A802031C722B7E303307A80703185B
:1076E000352B772B7E303307A807031CC82B1830A7
:1076F000B200A20DA30DA40DA50DA60DA70DB30DEF
:107700002C08A5022D08031C2D0FA6022E08031C11
:107710002E0FA7022E0DB304331C902B22149B2B8B
:107720002C08A5072D0803182D0FA6072E080318EF
:107730002E0AA7072210B20B792B2A1B221CBF2B63
:107740000310A50DA60DA70DB30D2C08A5022D083D
:10775000031C2D0FA6022E08031C2E0FA7022E0DB0
:1077600033040139A2070318A30A0319A40A031D4D
:10777000BF2BA40CA30CA20CA80A0319352BA91F1C
:10778000A4132408A7002308A6002208A50000349B
:107790002A15AA1FFF340130A800A701A601A501E0
:1077A000A90DA70CFF34AA15FF348030AE062708B8
:1077B0002E06B300A401AB0128082F02031CF82BEE
:1077C0002F08A2002808AF002208A8002E08A20057
:1077D0002708AE002208A7002D08A2002608AD0049
:1077E0002208A6002C08A2002508AC002208A5004B
:1077F0002F08031900342708A900A717AE172F0870
:107800002802AF0003192B2C08302F02031C212C57
:10781000AF002C08AB002D08AC002E08AD00AE0167
:1078200008302F02031C212CAF002C08AB002D08C0
:10783000AC00AD0108302F02031C212C2908A70041
:1078400000342F0803192B2C0310AE0CAD0CAC0C1C
:10785000AB0CAF0B242CB31F382CAB09AC09AD0912
:10786000AE09AB0A0319AC0A0319AD0A0319AE0A33
:107870002B08A4072C0803182C0FA5072D080318A4
:107880002D0FA6072E0803182E0FA707B31B512C88
:10789000031CCF2AA70CA60CA50CA40CA80FCF2A5A
:1078A000352B0318A02AA409A509A609A709A40A2B
:1078B0000319A50A0319A60A0319A70A8030A90605
:1078C000742AA401A3012708B3002608B2002508E2
:1078D000B1000830B400AD0C03187C2CB40B6B2C39
:1078E000B400AE0C03187A2CB40B712CA701A601BE
:1078F000A50100340310A02C03108B2CAD0C031C2D
:107900008B2C3108A50732080318320FA60733085D
:107910000318330FA707A70CA60CA50CA40CB40BD7
:107920007E2C0830B400AE0C031CA02C3108A50737
:1079300032080318320FA60733080318330FA707BE
:10794000A70CA60CA50CA40CA30CB40B932C003410
:10795000A401A301A2012708B3002608B20025084C
:10796000B1000830B400AC0C0318CC2CB40BB32C11
:10797000B400AD0C0318CA2CB40BB92CB400AE0C77
:107980000318C82CB40BBF2CA701A601A501003415
:107990000310062D0310F02C0310DB2CAC0C031C81
:1079A000DB2C3108A50732080318320FA60733086D
:1079B0000318330FA707A70CA60CA50CA40CB40B37
:1079C000CE2C0830B400AD0C031CF02C3108A507F8
:1079D00032080318320FA60733080318330FA7071E
:1079E000A70CA60CA50CA40CA30CB40BE32C08301C
:1079F000B400AE0C031C062D3108A507320803188D
:107A0000320FA60733080318330FA707A70CA60CDD
:107A1000A50CA40CA30CA20CB40BF92C0034A501EA
:107A20002808031900342708A4002608A3007F3083
:107A30002802B200B21B642D0F3CB300B200B21991
:107A4000412D0730B3057030B307BD300318013E38
:107A50008A00330A7025A605A71F0034A00023085A
:107A60002602031D342D00342009B200320AA60775
:107A70000319A70A031D0034A70CA60CA80F003495
:107A800084290730B3057030B307BD300318013EB9
:107A90008A00330A7025A705A601A71F0034A0009D
:107AA00023082602031D592D24082702031D592DE2
:107AB00000342009B200320AA707031C0034A70CC7
:107AC000A60CA80F00348429A71B6A2DA801A701C2
:107AD000A60100347F30A8008030A700A601003442
:107AE0008200FF34FE34FC34F834F034E034C03427
:107AF00080340034A51F003403147F30250503199A
:107B0000260C2708A900A71703110318A60A0319B2
:107B1000A70A031D902DA70CA60CA80A03198429F7
:107B2000A91FA7130034A5012808A71F0319932E26
:107B30002A08BE002A132808C3007E30C302A8000A
:107B4000F33025020430B300031C330F2602353016
:107B5000B300031C330F2702031C032E7F30AF003A
:107B6000AE01AD01AC01D5232808BA002708BB003F
:107B70002608BC002508BD008130AF002C30AE00C7
:107B80005130AD005030AC00D7233A08AF003B086D
:107B9000AE003C08AD003D08AC00E2228130AF00F1
:107BA0002330AE002430AD009630AC00D723280837
:107BB000B5002708B6002608B7002508B8003A081F
:107BC000A8003B08A7003C08A6003D08A50081309E
:107BD000AF000230AE00E130AD00B330AC00E222C5
:107BE0008130AF006B30AE005D30AD003930AC009D
:107BF000D7233508AF003608AE003708AD00380887
:107C0000AC004023592EA80A7F30AF00AE01AD0171
:107C1000AC01D523C3032808BA002708BB002608F7
:107C2000BC002508BD008130AF005730AE00DB300E
:107C3000AD003A30AC00D7233A08AF003B08AE00A5
:107C40003C08AD003D08AC00E2228130AF0064305A
:107C5000AE00B830AD000A30AC00D7232808B5001C
:107C60002708B6002608B7002508B8003A08A8007B
:107C70003B08A7003C08A6003D08A5008130AF00E6
:107C80001230AE007A30AD00CE30AC00E22282304D
:107C9000AF002430AE00FC30AD002230AC00D72362
:107CA0003508AF003608AE003708AD003808AC0024
:107CB00040233A08AF003B08AE003C08AD003D0849
:107CC000AC00E2222808BA002708BB002608BC0046
:107CD0002508BD00A7014308A600A61BA7099C20F4
:107CE000A5013A08AF003B08AE003C08AD003D08D6
:107CF000AC00D7232708C300A7179A30AE00203066
:107D0000AD009B30AC00A824A803A71B8C2EA40DAB
:107D1000A50DA60DA70DA803C31FA7133E1F003472
:107D20002A177A250034AA16FF3464302802B300DB
:107D3000B31BB22FA71BAD2E2808843C031C932E27
:107D4000031DBD2E27081A3C031C932E031DBD2EB8
:107D50002608213C031C932EBD2E2808843C031CBE
:107D6000932E031DBD2E2708973C031C932E031D45
:107D7000BD2E2608B83C031C932E2A08BE002A13E9
:107D8000B8277E302802031D392F271F002F7B3094
:107D9000AF005030AE006530AD00DC30AC00E22208
:107DA0007C30AF003130AE00E930AD003C30AC008B
:107DB000D7233A08AF003B08AE003C08AD003D08B1
:107DC000AC00E2227E30AF003B30AE00C430AD00EC
:107DD0009730AC00D7233A08AF003B08AE003C0810
:107DE000AD003D08AC00E2227E30AF007D30AE0039
:107DF000B430AD005430AC00D7234308A80700349A
:107E00007B30AF002F30AE003D30AD00B530AC0060
:107E1000E2227C30AF005730AE005130AD00F73079
:107E2000AC00D7233A08AF003B08AE003C08AD00D9
:107E30003D08AC00E2227E30AF003430AE00B330FB
:107E4000AD008130AC00D7233A08AF003B08AE004C
:107E50003C08AD003D08AC00E2227E30AF007F3030
:107E6000AE007E30AD000830AC00D7234308A80731
:107E700000347D302802031D762F7B30AF00133095
:107E8000AE005C30AD000C30AC00E2227C30AF00C4
:107E90006C30AE005230AD006130AC00D7233A08F0
:107EA000AF003B08AE003C08AD003D08AC00E2224C
:107EB0007E30AF003230AE000930AD009830AC00FB
:107EC000D7233A08AF003B08AE003C08AD003D08A0
:107ED000AC00E2227E30AF007F30AE00F230AD0069
:107EE0007D30AC00D7234308A80700347A30AF00B8
:107EF0007730AE00D430AD000830AC00E2227C30E8
:107F0000AF007530AE003030AD00A030AC00D723EC
:107F10003A08AF003B08AE003C08AD003D08AC009D
:107F2000E2227E30AF003130AE007430AD00A130BF
:107F3000AC00D7233A08AF003B08AE003C08AD00C8
:107F40003D08AC00E2227E30AF007F30AE00FF3053
:107F5000AD00FB30AC00D7234308A8073E1F003418
:107F60002A177A2D7F30A800A701A601A5010034A9
:107F70002708BB00A7172708AE002608AD00D4309D
:107F8000A7009A30A6007830A5006124A80AA80AA4
:107F9000A71BCF2FA40DA50DA60DA70DA803BB1FD2
:107FA000A7132808AF002708AE002608AD00250853
:107FB000AC000F252808BA002708BB002608BC0023
:107FC000F9202608C3003A08A8003B08A7003C088F
:107FD000A600A5018030A706D7232808BA002708E5
:0C7FE000BB002608BC002508BD000034D2
:020000040001F9
:080000000000000000000300F5
:02000E00840963
:02001000FF1CD3
:10E000000500020040000100050055008400680082
:10E0100066007800320014004B0000000000000091
:06E04000040012000000C4
:06E04A00310020000F0070
:0CE050000F000000120014000D00000082
:02E05E001200AE
:10E0600013001B002900000004001200010004003E
:10E070001200010004001200010015000600140047
:10E08000150001000500060001000B0002001C0045
:10E0900014000800070001000B0002001C0014001F
:0AE0A0000800070001000C0000005A
:02E0CE0016003A
:10E0D0001300010020000F000F00310001000300B9
:04E0E0000C00000030
:0CE13400120014000D0001001500160080
:02E140000000DD
:06E19A00120013001B003F
:10E1A000290001000500060001000B0002001C0010
:0CE1B00014000800070001000C00000033
:00000001FF
